:020000001028C6
:080008008B139200030E91001E
:1000100009280000110E8300920E120E8B170900A2
:100020008316093085000030860083128501860121
:100030003628C4202708A71B23282708970016085E
:10004000B5207C2019281F30270596001928472045
:100050001D089D171D08ED201E08ED20B52027283E
:1000600011309600003097007C2035284720B720BB
:100070001D08031D3628103096001E089700113CFD
:1000800003194528013C031D36287C20362805111C
:10009000051C4728B9209B019C010D309A00BB200C
:1000A0009B0D9C0D1B10051C1B146B20B920BB2045
:1000B0009A0B50281B089E001E139E139B0D9C0D2F
:1000C0009B0D9C0D1C089D009D131D139D121C1F54
:1000D0001E171E0808000930980020309900990B5F
:1000E0006F28051876281B1C080078281B180800A4
:1000F000980B6D2805150800812088208E209720F8
:100100000800A920171B8628A9200800AC20080099
:10011000930A131CA9201318AC2008000530950081
:1001200016089400940D940D940D9F20080006303D
:10013000950017089400940D940D9F200800940DCD
:100140000318A428AC20A528A920950B9F2885106A
:100150000800B220AF200800AF20B22008008514AC
:10016000BB2008008510BB2008002D30BC28FF30C4
:10017000BC280930BC28123098000F309900990B28
:10018000BF28980BBD280800A80108309800851DDD
:10019000C428E820851DC428E02085190310851D8A
:1001A0000314A80C980BCC28E0208519C428E02063
:1001B0008519C4282808A70008000F309900E228F4
:1001C0000F309900000000000000990BE2280800A1
:1001D0000F309000900BEA280800A8000830980023
:1001E0000511DD200515DD20A80C03180511031CE1
:1001F0000515DD20980BF4280511DD200800FA30E4
:100200009F00032108006E30A000000000000000E5
:10021000000000000000A00B05299F0B03290034FB
:00000001FF
